:03200000022100BA
:03202B00022FF889
:1021000075BF0143B70843B70453B6F743B6047924
:1021100000780AD9FED8FC785643B602D8FEE5B658
:1021200030E0F475BB9853B70F43B7A053B7FB43E8
:10213000B7027864D8FEE5B730E0DC53B7F775BF77
:102140000078FFE4F6D8FD90F0007F007E06E4F012
:10215000A3DFFCDEFA75819F0221960221DBE49366
:10216000A3F8E493A34003F68001F208DFF480298A
:10217000E493A3F85407240CC8C333C4540F442079
:10218000C8834004F456800146F6DFE4800B010268
:10219000040810204080902A3BE47E019360BCA399
:1021A000FF543F30E509541FFEE493A360010ECFB6
:1021B00054C025E060A840B8E493A3FAE493A3F8E0
:1021C000E493A3C8C582C8CAC583CAF0A3C8C582A0
:1021D000C8CAC583CADFE9DEE780BEAEB4EE7002CE
:1021E0007F01122B73E4F5BF7581C0D280D2B67D1A
:1021F00002FF123F7D7B017AF079EE123BFA90F1FB
:1022000016EEF0A3EFF07B017AF079541235CE127E
:1022100030FF122E661242C0122EE080F27C0112B4
:102220002DAE7F027E002202256FE86480F8E9333C
:10223000E83360110460F0ED33EC337009E8FCE939
:10224000FDEAFEEBFF220460DED3EB9FEA9EE99DF0
:10225000E8C2E78CF0C2F795F0400CE8CCF8E9CD85
:10226000F9EACEFAEBCFFB12253A85D0F05804708C
:102270000320D5B3E80470075002B2D50225799245
:10228000D5EC0460F7E4CCC0E0C398F8603B941848
:102290006008400DD0E0FB022551E4FBFAC9FC8048
:1022A00028E830E406E4C9FBE4CAFCE830E305E4CE
:1022B000C9CACBFCE854076010F8C3E913F9EA1364
:1022C000FAEB13FBEC13FCD8F130F52FC3E49CFCC4
:1022D000EF9BFFEE9AFEED99FDD0E0FBEF4E4D4CEB
:1022E000701222DB03022576EC2CFCEF33FFEE3379
:1022F000FEED33FDED30E7EB022551EF2BFFEE3A1B
:10230000FEED39FDD0E0FB50130BBB000302257935
:10231000ED13FDEE13FEEF13FFEC13FC022551EC61
:102320004D6011E8497017ED33EC3304600DE4FCA7
:10233000FFFEFD22E933E8330470F802256F122511
:102340003A58046009E4CC2481500628500902253B
:1023500079284003022576C0E0EB4A7044B9800634
:10236000D0E0FB022565EF4E701CBD8008EBFFEA54
:10237000FEE9FD80EBE98DF0A4FEE5F0022408E91A
:10238000CDF9EAFEEBFFEF89F0A4FCE5F0CE89F091
:10239000A42EFFE435F0CD89F0A42DFEE435F080C5
:1023A00067EF4E7005BD80D780C3EF8BF0A4ACF013
:1023B000EE8BF0A42CFCE435F0F8EF8AF0A42CE5C9
:1023C000F038FCE433CB8DF0A42CFCE5F03BF8EEC8
:1023D0008AF0A42CFCE5F038F8E433CF89F0A42C83
:1023E000FCE5F038CF3400CE89F0A42FFFE5F03EB5
:1023F000FEE433C98DF0A42EFEE5F039CD8AF0A4B9
:102400002FFFE5F03EFEE43DFD33D0E0FB50070B2F
:10241000BB000F022579EC2CFCEF33FFEE33FEED11
:1024200033FD022551022579EC5D046005E859046D
:10243000700302256F12253A580460F6EC4860F2EA
:10244000EC7004FDFEFF22C860DB2481C85009C384
:1024500098600250060225769850CAF582E9294B09
:102460004A7005AB8202256575F0007C1A7880C33E
:10247000EF9BEE9AED99400DC3EF9BFFEE9AFEEDB8
:1024800099FDE842F0DC23ACF0D0E0FFD0E0FED0D4
:10249000E0FDAB8220E7101BEB60BAEC2CFCEF33C5
:1024A000FFEE33FEED33FD022551E803F830E7057A
:1024B000C0F075F000EF2FFFEE33FEED33FD40B8B6
:1024C00030E7C280AA75F020800E75F01080057587
:1024D000F0087D007E007F003392D530D5031226B0
:1024E000BBEC334010EF33FFEE33FEED33FDEC3346
:1024F000FCD5F0ED22E5F0247EA2D513CC92E7CDF9
:10250000CEFF22EDD2E7CD33EC3392D524814006C5
:10251000E4FFFEFDFC22FCE4CFCECDCC24E0501144
:1025200074FF80EDC3CC13CCCD13CDCE13CECF131F
:10253000CF0470F030D5DE0226BBE9D2E7C933E81C
:1025400033F892D5EDD2E7CD33EC33FC5002B2D55F
:1025500022EC30E7100FBF000C0EBE00080DBD00CE
:10256000040BEB6014A2D5EB13FCED92E7FD227493
:10257000FFFCFDFEFF22E480F8A2D574FF13FC7D72
:1025800080E480EFBB010689828A83E0225002E763
:1025900022BBFE02E32289828A83E49322BB010CE0
:1025A000E58229F582E5833AF583E0225006E925A4
:1025B00082F8E622BBFE06E92582F8E222E58229BE
:1025C000F582E5833AF583E49322BB010FF8E582B7
:1025D00029F582E5833AF583E028F0225009C58287
:1025E00029F8E58226F622BBFE09C58229F8E225F4
:1025F00082F222F8EA2583F583E9932822BB0106BB
:1026000089828A83F0225002F722BBFE01F322F86E
:10261000BB010DE58229F582E5833AF583E8F022D6
:102620005006E92582C8F622BBFE05E92582C8F2DC
:1026300022BC000BBE0029EF8DF084FFADF022E438
:10264000CCF875F008EF2FFFEE33FEEC33FCEE9D77
:10265000EC984005FCEE9DFE0FD5F0E9E4CEFD229E
:10266000EDF8F5F0EE8420D21CFEADF075F008EF29
:102670002FFFED33FD4007985006D5F0F222C398A6
:10268000FD0FD5F0EA22A3F8E0C5F025F0F0E582D1
:10269000158270021583E0C838F0E822BB010A8970
:1026A000828A83F0E5F0A3F0225006F709A7F0191B
:1026B00022BBFE06F3E5F009F31922C3E49FFFE411
:1026C0009EFEE49DFDE49CFC22EB9FF5F0EA9E4219
:1026D000F0E99D42F0EC6480C864809845F022EBFC
:1026E0009FF5F0EA9E42F0E99D42F0E89C45F02219
:1026F000E8600FECC313FCED13FDEE13FEEF13FFC8
:10270000D8F122E8600FEFC333FFEE33FEED33FD67
:10271000EC33FCD8F122BB010789828A83022A1399
:102720005005E9F8022A07BBFE05E9F8022A1F89CD
:10273000828A83022A2BECF0A3EDF0A3EEF0A3EF44
:10274000F022A8828583F0D083D0821227591227E5
:1027500059122759122759E473E493A3C583C5F08E
:10276000C583C8C582C8F0A3C583C5F0C583C8C5E5
:1027700082C822E3F5F009E208B5F06BDFF5806767
:10278000E3F5F009E608B5F05EDFF5805A87F00959
:10279000E608B5F052DFF6804E87F009E208B5F0A2
:1027A00046DFF6804288828C8387F009E0A3B5F08B
:1027B00036DFF6803288828C8387F009E493A3B5F4
:1027C000F025DFF5802188828C83E3F5F009E0A312
:1027D000B5F014DFF5801088828C83E3F5F009E40E
:1027E00093A3B5F002DFF402289E808780E98090F1
:1027F00080D4803C8015806C807C809D80B7808DEB
:1028000080A3804F8072803A0228AA89828A8363DB
:10281000A20188828C8363A201E493F5F0A363A2F2
:1028200001E493A363A201B5F074DFEDDEEB806EEB
:1028300089828A83E493F5F0A3E208B5F060DFF4BF
:10284000805C89828A83E0F5F0A3E608B5F04FDF6B
:10285000F5804B89828A83E0F5F0A3E208B5F03E6B
:10286000DFF5803A89828A83E493F5F0A3E608B520
:10287000F02CDFF480288002805389828A8363A24F
:102880000188828C8363A201E493F5F0A363A20123
:10289000E0A363A201B5F006DFEEDEEC80007FFF6F
:1028A000B5F0020F2240027F012289828A8363A24F
:1028B0000188828C8363A201E0F5F0A363A201E0AA
:1028C000A363A201B5F0D7DFEFDEED80D189828A64
:1028D0008363A20188828C8363A201E0F5F0A36385
:1028E000A201E493A363A201B5F0B3DFEEDEEC80B6
:1028F000AD88F0EF60010E4E60AFED2402B404002D
:10290000509CF582EB2402B40400509223234582AC
:10291000239027EA73E709F608DFFA8046E709F211
:1029200008DFFA803E88828C83E709F0A3DFFA8013
:1029300032E309F608DFFA8076E309F208DFFA806D
:102940006E88828C83E309F0A3DFFA806289828A31
:1029500083E0A3F608DFFA805689828A83E0A3F237
:1029600008DFFA804A80D280FA80C680D4806580F1
:10297000F28031801080A680EA809A80A880DA8078
:10298000E280CA803189828A8363A20188828C8333
:1029900063A201E493A363A201F0A363A201DFF3A6
:1029A000DEF1800B89828A83E493A3F608DFF9ECD9
:1029B000FAA9F0EDFB2289828A8363A20188828CC6
:1029C0008363A201E0A363A201F0A363A201DFF489
:1029D000DEF280DB89828A83E493A3F208DFF98048
:1029E000CE88F0EF60010E4E60C588F0ED2402B491
:1029F000040050BBF582EB2402B4040050B1232341
:102A000045822390296573E6FC08E6FD08E6FE088A
:102A1000E6FF22E0FCA3E0FDA3E0FEA3E0FF22E24C
:102A2000FC08E2FD08E2FE08E2FF22E493FC7401E8
:102A300093FD740293FE740393FF2258F00000008C
:102A40000000000000000000000000000000000086
:102A500000000000000044F0470000000042F03C8D
:102A60000000C100C10142F03A03E848F03E000016
:102A700000000000000048F04B00000000000000D3
:102A80000048F021000000000000000048F0540061
:102A90000101000000000048F029000000000000D3
:102AA000000050F06D000000000000000000000079
:102AB000000000000050F05D000000000000000079
:102AC000000000000000000048F0190000000000B5
:102AD00000000048F032000000000000000041F05B
:102AE000310050F07E0000000000000000000000F7
:102AF000000000000041F0460041F0180041F07D68
:102B000000C102C10341F05C0041F0530048F0E60F
:102B100000000000000000004AF0DC00000000009F
:102B20000000000000008E198F188C1C8D1BE4F52E
:102B30001DF51EF51FC0D0C0E0C0F043D01812DF55
:102B4000F94008D0F0D0E0D0D0D322D0F0D0E0D0FF
:102B5000D0C3228F18C0D0C0E0C0F043D01812DF1D
:102B6000F64008D0F0D0E0D0D0D322D0F0D0E0D0E2
:102B7000D0C32275BF0175BA10E4F5BFB1BE123FD4
:102B8000F6D13B1240087196F1EDE4F5B8F5B9F5D0
:102B9000F8F5F9D2AF2275DA0075D97175DC01E567
:102BA000DC30E00553D8FE80F675DA0075D9807503
:102BB000DB4975D815E5D820E1FB75D804D132E59D
:102BC000D820E1FBD132E5D820E1FB75DB4B75DC89
:102BD0003A75D835E5D820E1FB75DD6075D845E557
:102BE000D820E1FBE4F5DBF5DCF5DD75D871E5D83F
:102BF00020E1FB75DA0075D9C075DB4175D815E5A4
:102C0000D820E1FB75B202439002439102E4F5B291
:102C1000439102F5DA75D9717F02FE7D0812221DFB
:102C20007D0512221D7D0612221D7D0712221D7DAB
:102C30000912221D7D0A12221D7D0B12221D7D0C00
:102C400012221D7D0D7C01B1AE75DA0475D92FD12C
:102C50002BB1A67F037E007D007CE0B18ED119B13F
:102C6000A87F007E05B197D10B75D937D122B1A8C5
:102C70007F01B188D119B1A87F007E06B197D10B31
:102C800075D93FD12BB1A67F02B188D119B1A87FE8
:102C9000007E07B197D10B75D947D122B1A87F0229
:102CA0007E007D007CF1B18ED119B1A87F007E0835
:102CB000B197D10B75D94FD122B1A87FF07EFF7D9E
:102CC000FF7CFFB18ED119B1A87F007E09B197D1E9
:102CD0000B75D957D122B1A87F027E007D007CF40C
:102CE000B18ED119B1A87F007E0AB197D10B75D9E9
:102CF0005FD12BB1A67F04B188D119B1A87F007E26
:102D00000BB197D10B75D967D122B1A87F03B188D8
:102D1000D119B1A87F007E0CB197D10B75D96FD1B5
:102D20002BB1A67F017E007D007CF4B18E7FFF7EFB
:102D3000FF7DFF7C1FB1A87F007E0DB1977F007ED5
:102D4000007D007C08B16175DA0075D980E4F5D8A2
:102D5000E5D820E1FB53DBBE75D811E5D820E1FBB7
:102D60002290F0AC12273690F0AFE0F5DB90F0AE99
:102D7000E0F5DC90F0ADE0F5DD90F0ACE0F5DE756F
:102D8000D8F1E5D820E1FB227E007D007CF5B16121
:102D900075D8087F007E007D007C00B16175D80881
:102DA0007F007E007D007C00B16175D80822B16192
:102DB00075DC01E5DC30E00553D8FE80F62275B203
:102DC0000375800875B2017580FE7586EFE4F5B273
:102DD00075860D75800C75B203F59075B20175900E
:102DE000DF7591BFF5B275916075B20375B03C7532
:102DF000B20175B03F75B1FCF5B275B1FC75B201A9
:102E0000F5C875C908F5B275C908227F007E007D36
:102E1000007C08B16175DA04227FFF7EFF7DFF7CB4
:102E20003F227F007E007DA87C0E227F007E007DF9
:102E3000A022E4F5DBF5DC75D83522D15975BCDB71
:102E400043BB0443BB03538FFE75BF0175BBABF59A
:102E5000BF22D15953BBFB80ED75BF0175BB9BE40D
:102E6000F5BF438F012290F090743FF0C2AFE5D8D8
:102E700020E1FBC0D9C0DAC0DBC0DCC0DDC0DE753C
:102E8000BF80D1D9E4F5D8E5D820E1FB90F08EE5FC
:102E9000DBF0A3E5DCF090F08EE030E50271969077
:102EA000F08EE0FF5407600690F0907438F0D1D9AE
:102EB00090F090E05FF4F5DB90F08FE0F4F5DC75D6
:102EC000D831E5D820E1FB75BFC0D0DED0DDD0DC45
:102ED000D0DBD0DAD0D9D2AF2275DA0075D9812211
:102EE0007F05123885EF7002E196F1F17F051242FD
:102EF000F890F0A5F090F099E090F0A4F090F09A9E
:102F0000E090F0A3F090F09BE090F0A2F090F09CA5
:102F1000E090F0A9F090F09DE090F0A8F090F09E85
:102F2000E090F0A7F090F09FE090F0A6F07F0512FF
:102F3000384FC2AFC2C2D15290F0A2E064AA700F63
:102F4000A3E064AA70097D017F55123A228079902E
:102F5000F0A2E06433703FA3E064337039F5BFF54D
:102F6000BCFD7C03FFFE7126F197E4FFEFC39420C4
:102F700074809480500974802FF8E4F60F80ED7807
:102F800080761175836FE4F5827F807153F1977DB0
:102F9000047F55123A2222538FFEE4F5BFFFEFC3A0
:102FA0009432748094805020E4FEEEF1E55016E4F3
:102FB000FDEDF1E5500CE5BC30E20453BCFB220D05
:102FC00080EF0E80E50F80D675BF0175BB9B438FE8
:102FD0000143BB0475BCFF43BB03538FFE75BBAB02
:102FE000E4F5BF80FEC394FF748094802243A82040
:102FF000227B017AF0798E22C0E0C0F0C083C082CB
:10300000C0D075D00063A201C083C08263A201C09A
:1030100000C001C002C003C004C005C006C00790C4
:10302000F0DB743FF0E5D820E1FBC0D9C0DAC0DBAB
:10303000C0DCC0DDC0DE75BF8030C704C2C711C4AC
:10304000E5B65401604A53B6FE122ED975D800E594
:10305000D820E1FBAFDBAEDCEF30E51B30E70A90B8
:10306000F05C7480F0EF547FFFEF30E60A90F05C84
:103070007440F0EF54BFFF122ED990F0DBE05FF404
:10308000F5DBAF06EEF4F5DC75D831E5D820E1FBD1
:1030900075BFC0D0DED0DDD0DCD0DBD0DAD0D9D067
:1030A00007D006D005D004D003D002D001D00063F1
:1030B000A201D082D08363A201D0D0D082D083D0AD
:1030C000F0D0E03230002490F03DE004F070069043
:1030D000F03CE004F090F03A11F890F03DE09F9061
:1030E000F03CE09E400CC200E48004E490F03CF030
:1030F000A3F022EDF090F0AAE0FEA3E0FFC3227857
:103100008E7CF07D017BFF7A0079087E007F1412AF
:1031100029E1E490F0A212429BF0A312429BF07FBF
:103120000B123885EF6051122FF17F0B1242F8908D
:10313000F02CF090F099E090F02BF090F09AE09065
:10314000F02AF090F09BE090F029F090F09CE09055
:10315000F030F090F09DE090F02FF090F09EE09035
:10316000F02EF090F09FE090F02DF07F0B12384F92
:103170007B017AF07929B1CE7F0D123885EF600E90
:10318000122FF17F0D910A7F0D12384FD2037F0766
:10319000123885EF7002416D122FF17F071242F84D
:1031A00090F00BF090F099E090F00AF090F09AE037
:1031B00090F009F090F09BE090F008F090F09CE027
:1031C00090F00FF090F09DE090F00EF090F09EE007
:1031D00090F00DF090F09FE090F00CF07F07123827
:1031E0004F90F018E004F090F00CE090F046F09072
:1031F000F00912430090F00812426DD31226C95014
:103200000312430B1242D712425E7D3C1242A6903B
:10321000F0431242501242A490F04111F3941EEE7A
:10322000940090F0404005741EF08002EFF090F0A2
:103230000B12430090F00A12426DC31226C95003CC
:1032400012430B1242D712425E7D3C1242A690F00E
:10325000501242501242A490F04E11F3941EEE947C
:103260000090F04D4005741EF08002EFF07B017A73
:10327000F07931123A6D300002615AD2007B017A46
:10328000F0792171B07F09717D90F0EAEFF07F0A4B
:10329000717D90F0E8717990F0E7717990F0EBEF43
:1032A000F07F0C717D90F0E9EFF012403790F07DE7
:1032B000E0FF90F018E06F7049C20290F06EE044B9
:1032C00001F0E04402F0E04404F0E04410F0E04497
:1032D00020F090F05DE04401F090F06EE04408F0E2
:1032E00090F05DE04410F03003227B017AF0796DBC
:1032F0007F0A1239037B017AF0795D7F0812390366
:10330000800AD20290F018E090F07DF0124096A270
:1033100092E43354011242CE54FEFDEC12428EA2CE
:1033200094B3E433540125E0FFE433FE1242CF545A
:10333000FD12428BA202E4FE3354017802C333CE65
:1033400033CED8F91242CE54FB12428B30030B7BA2
:10335000017AF079E67F0C12390390F05CE0FF64AB
:10336000406005EF6480701090F05CE090F053F0E6
:10337000122B96E490F05CF022EFF07F0BAD071279
:103380004167AF05F1E81241487FA3F1E81241F629
:10339000C2041241CBC20571A500D205F1EE0000B6
:1033A000000000D205E4F5B2438608A2059283220C
:1033B0007F08717D12422BEF1225FD7F07717DEF93
:1033C000541FFF12422B900001EF12260F7F0512AF
:1033D000423A900002EF12260F7F0412423A900008
:1033E00003EF12260F7F06717DEF54079000041241
:1033F000260F7F03124224900005EF12260F7F0252
:10340000124224900006EF02260F123B5BE5D82003
:10341000E1FBC0D9C0DAC0DBC0DCC0DDC0DE1242D7
:10342000B72400123845E4F5D8E5D820E1FBB1C255
:10343000E5DE1225FD1242B72404123845E4F5D822
:10344000E5D820E1FBB1C290000DE5DB12260F901C
:10345000000CE5DC12260F90000BE5DD12260F9024
:10346000000AE5DE12260F75D804E4F5D8E5D82069
:10347000E1FBB1C2900011E5DB12260F900010E5D0
:10348000DC12260F90000FE5DD12260F90000EE5EE
:10349000DE12260F90F0ACE012383FE4F5D8E5D804
:1034A00020E1FBE5DC30E30F90F0ADF1F6240112F2
:1034B00042F144081225FD124316E5D820E1FBE550
:1034C000DE30E554B1C2900005E5DB12260F900016
:1034D00004E5DC12260F9000031242AD90000212A8
:1034E000260F123B54124316E5D820E1FBB1C290DF
:1034F0000009E5DB12260F900008E5DC12260F908C
:1035000000071242AD90000612260FE92401124274
:10351000F144041225FD806D124327B1C2900005CD
:10352000EF1242AF90000412260F900003E412261F
:103530000F900002E412260F9000041242E42404CB
:10354000B1B4900005EF1225CA123B54124316E5A0
:10355000D820E1FB124327B1C2900009EF1242AF1D
:1035600090000812260F900007E412260F90000624
:10357000E412260F9000081242E42408B1B490002F
:1035800009EF1225CA1242B72402123845E4F5D8D1
:10359000E5D820E1FBB1C2900013E5DD12260F90C3
:1035A0000012E5DE12260FD0DED0DDD0DCD0DBD07D
:1035B000DAD0D922F9E43AFA1225841313543F12CF
:1035C00025FD90F0ADE0FBA3E0FAA3E0F92290F036
:1035D000AF123B61E4A3F078B37CF07D017BFF7A0E
:1035E00000791CFE7F081229E1F1F34A4B7002C1F9
:1035F000BC78B37CF07D0190F0AFB1C7123A669011
:10360000F0B3E0FF7B63E4FDD1CCEFF0A3E0FF7B00
:103610000C0DD1CCEFF0A3E0FF7B1FD1CCEFF0A3DA
:10362000E0FF7B171DD1CCEFF0A3E0FF7B06D1CCF0
:10363000EFF0A3E0FF7B3BD1CCEFF0A3E0FFD1CCD8
:10364000EFF090F0AFB1C5122584FFD1DDAD077F5B
:1036500008F1DAB1C5900001F1E0541FFD7F07F1D8
:10366000DAB1C5900002F1E0543FFD7F05F1DAB117
:10367000C5900003F1E0543FFD7F04F1DAB1C5903D
:10368000000412259D5407FD7F06F1DAB1C59000B4
:1036900005F1E0547FFD7F03D1BD7F02717DEF54C2
:1036A0008090F0B2F090F0AFB1C5900006F1E05418
:1036B0007FFF90F0B2E04FFD7F02D1BD22AC071238
:1036C0004167AF04F1E8AF05F1E86195EFC39D50A4
:1036D00003AF0522EFD39B4003AF032222EF75F027
:1036E0000A84C454F0FEEF75F00A84E5F04EFF2220
:1036F00090F0AF123B6178B27CF07D017BFF7A00E5
:103700007924123A6678BA7CF07D017BFF7A0079E1
:103710002C123A66E490F0C2F0FCF1F34A4B6016CA
:1037200090F0AFA3A3E0F9123B4E700D123B48702E
:1037300008123B4270037F01227B017AF079B2715B
:10374000B090F0AFB1C5123B4EFF90F0B7E02F90B4
:10375000F0BFF0E0C3943C74809480400AE024C43D
:10376000F090F0C27401F0123B48FF90F0B5E02FEA
:10377000FF90F0C2E02F90F0BDF0E0C39418748089
:1037800094804006E024E8F07C01123B42FF90F078
:10379000B4E02F2C90F0BCF0E0C3941F74809480B0
:1037A0004003741FF0E490F0BEF090F0BC12431D93
:1037B0007F0BD1BDA312431D7F0AD1BD7D807F0C3D
:1037C000D1BD90F0BFE0FFD1DDEF547FFD7F09D187
:1037D000BD7D027F01D1BD7F0022D1BD90F0AF221F
:1037E00012259DFFD1DDEF2212419B02416DA20502
:1037F00092822290F0AFE0FBA3E0FAA3E022E4FD86
:10380000E5D820E1FBC0D9C0DAC0DBC0DCC0DDC038
:10381000DE113EE4F5D8E5D820E1FBE5DC5401708B
:103820000EF5DC75DB20117DE5D820E1FB7D01D0B4
:10383000DED0DDD0DCD0DBD0DAD0D9AF0522EF7519
:10384000F008A42407FFE5F03404F5DA8FD922E567
:10385000D820E1FBC0D9C0DAC0DBC0DCC0DDC0DEEF
:10386000113E75DC0075DB08E4117DE5D820E1FB35
:10387000D0DED0DDD0DCD0DBD0DAD0D922F5DEF559
:10388000DD75D8F122E4FDE5D820E1FBC0D9C0DA2E
:10389000C0DBC0DCC0DDC0DE113EE4F5D8E5D820D9
:1038A000E1FBE5DB30E3027D01D0DED0DDD0DCD012
:1038B000DBD0DAD0D9AF052290F0B8EFF0A3122711
:1038C0004200000000E47F707E17FDFC90F0B9120A
:1038D000413CC31226DF502A90F0B8E0FF1237FEB9
:1038E000EF701F1242C090F0B9E0FCA3F1E5240193
:1038F000FFE43EFEE43DFDE43CFC90F0B9122736C7
:1039000080C322715B78B07CF07D017BFF7A007907
:103910000051661235C212258490F0B2F090000179
:1039200012259D90F0B3F0714290F0B0F071489084
:10393000F0B1F090000412259D90F0B6F0714E9019
:10394000F0B7F090000612259D90F0B4F0900007BB
:1039500012259D90F0B5F090F0ACE0FF11B890F01A
:10396000ACE0FF7B017AF079B031B990F0ACE0FFC8
:10397000E5D820E1FBC0D9C0DAC0DBC0DCC0DDC0C7
:10398000DE113EE4F5DCF5DB75DE0775DD2075D86C
:10399000F1E5D820E1FBD0DED0DDD0DCD0DBD0DA21
:1039A000D0D9223003127F0611B87B017AF079005A
:1039B0007F0631B97F06317022E5D820E1FBC0D9FE
:1039C000C0DAC0DBC0DCC0DDC0DE113EE4F5DCF5F2
:1039D000DBF5DE75DD0875D8F1E5D820E1FB715423
:1039E00075D808712AE5D820E1FB75D8047404293C
:1039F000F9E43AFA712AE5D820E1FB75D80475D8C4
:103A00000475DC0075DB4075DE0075DD2075D8F1CE
:103A1000E5D820E1FBD0DED0DDD0DCD0DBD0DAD0C1
:103A2000D92290F0AAEFF0A3EDF078AC7CF07D0104
:103A30007BFF7A007934516690F0AAE090F0AFF005
:103A400090F0ABE090F0AEF07B017AF079AC7F09BA
:103A500031B97F0931707F0901B878197CF07D0197
:103A60007B017AF0794B7E007F080229E190F0AC6F
:103A7000716190F0AC1235C512258414601E14607B
:103A80006B24026002612230020971231236F05168
:103A90005A802D90F0AC1235C5E4611F124243509C
:103AA00002804F78197CF07D0171237E007F08121F
:103AB00028F1EF3395E04F6011515A71231236F01F
:103AC00090F0AC1235C57401805590F046E0FF646B
:103AD000016005EF6402700A90F0AC1235C5740203
:103AE000803D90F0AC1235C57401803390F046E013
:103AF00070257B017AF079541235CE7B017AF0790A
:103B00003E1236F0C280D296C2B690F0AC1235C5E5
:103B1000E41225FD02402390F0AC1235C574021268
:103B200025FD227B017AF0794B22122716E48EDCE8
:103B30008FDB12271678101226F08EDE8FDD75D8F7
:103B4000F12290000202259D90000302259D900025
:103B50000502259D75D80875D8082290F0ACEFF0C5
:103B6000A3EBF0A3EAF0A3E9F02290F09C7161B11D
:103B700051EF7002FF227FCC71A57F4ED18390F070
:103B80009CD19C122584FF71A590F0A0E004F070F8
:103B90000690F09FE004F0C390F0A0E09403F1EDF4
:103BA00040DC7F0122AC07E4FBEBB1FB5014A8031F
:103BB000EC088003A2E713D8FB5401FAFF71C30B92
:103BC00080E722AD07D17A7F02FE71E7AF05EF33C0
:103BD00095E0FEEF64014E7002D2B57F197E007150
:103BE000E7D2B57F057E00D3EF9400EE9400400944
:103BF0000000EF1F70011E80EE2290F08E7161E4D4
:103C0000A3F078937CF07D017BFF7A00793CFE7F06
:103C1000051229E1E490F0D8F0A3F0A3F0B151EF40
:103C20007003FEFF227FF071A5E490F092F090F017
:103C300092E0B1FB4002A100E4FAEAB1FB4002814C
:103C4000CAD1BCEF5403FF90F0D8E0FEC313F0EFED
:103C500064027007FFB132E4F0806CEF640170071A
:103C6000B1297401F08060EF6002A12590F092E02C
:103C700075F008A42A04FC90F091E0F9B18BE0FB08
:103C8000ECD39B4012E4FFB132E4F090F091E004F9
:103C9000F0B18BECF08030ECC39B5017B134E0FFF7
:103CA0005401C43333335480FE90F0D8E04EF071A9
:103CB000C38014749329B18DE06C700BB129740129
:103CC000F090F091E014F00A813A90F0D8F1E578A4
:103CD00003C333CE33CED8F9FF90F08E1237F62FD0
:103CE000F9EA3EFA90F092E07E0029F9EE3AFAED18
:103CF0001225FDE490F0D8F090F092E004F0812ECF
:103D000090F0DAE004F0700690F0D9E004F090F062
:103D100091E0B18BE0600ED172C39405EE648094A3
:103D2000805002811DD172FF2290F0D8E04480F0D3
:103D30007F0171C390F092E075F008A42AF582E447
:103D400035F0F583E5822498F582E58334F0F58338
:103D500022E4FDFCD17B7FF0D18D7F28D13EFBEBAF
:103D60006019C3ED9411EC64809480500E7F057E41
:103D700000D13FFB0DBD00010C80E47FC87E0071C7
:103D8000E7AF03EB7F0160027F00222493F582E41A
:103D900034F0F5832290F0C37161A3EDF0B151EFDF
:103DA0007002FF227F5571A5E4F9E9B1FB50229022
:103DB000F0C6E075F008A424EEF582E434F0F58353
:103DC000E58229F582E43583F583E0FF71A509805A
:103DD000D97FBE71A5E490F0C7F090F0C7E0C3941E
:103DE00009748094805010D15AD199EF1225FD901A
:103DF000F0C7E004F080E37F0122EEC394087480F2
:103E000094802290F09C7161B151EF7002FF227F8B
:103E1000CC71A57FBED183D15A90F09CD19CEF127A
:103E200025FD90F0A0E004F0700690F09FE004F013
:103E3000C390F0A0E09409F1ED40DC7F0122FE7117
:103E4000E7A2B5E43322D17A7F01D18D7F03D13E41
:103E5000FD7F1B7E0071E7AF0522E4FCFBEBB1FBAD
:103E6000500DD1D98002C333D8FC4CFC0B80EEAF8F
:103E7000042290F0D9E0FEA3E022E4F5B243B120A1
:103E8000C2B52271A5E490F09FF0A3F022FE71E785
:103E9000D2B5E4F5B253B1DF2290F0C3E0FBA3E466
:103EA00075F001122686A9F0FA22B151EF7002FFD7
:103EB000227FCC71A57F4471A57F0122E4FCFBEB3E
:103EC000C3940274809480500DD1D98002C333D83A
:103ED000FC4CFC0B80E9AF0422D146A803EF08227A
:103EE00090F0C37161A3EDF0E4FE90F0C6E0FD1424
:103EF000F0ED6031D19912258490F0C7F0E4FFEF26
:103F0000B1FB50E690F0C7E0FD6E30E00AEE6418B9
:103F1000C3134480FE8004EEC313FEEDC31390F080
:103F2000C7F00F80DAAF062290F0B4716190F0C054
:103F30007401F0A374F0F0A374B7F07B017AF0F988
:103F4000B195EF7002FF227B017AF079B77D08D13D
:103F5000E090F0BFE06F60037F002290F0C0123568
:103F6000C590000112259DFE122584FDEDFF90F005
:103F7000B41235C5EE8FF012269C7F012290F08E90
:103F8000EFF0A3EDF090F0997401F0A374F0F0A3BA
:103F90007490F07B017AF0F9D103EF7002FF227B7D
:103FA000017AF079907D08D1E090F098E06F60039D
:103FB0007F002290F0991237F624061242F154FC49
:103FC000FF1225FD90F08FE04F1225FD54E3FF1204
:103FD00025FD90F08EE04F1225FD7B017AF079945B
:103FE000716A7F0122E0FDA3E0FEA3E02290F09F32
:103FF000E0648094802275C43075C5F875C2307550
:10400000C3F8E4F5C1D2C22275BF0175B41375B50A
:104010000275BF03E4F5BBF5BF43A80175880175C0
:10402000B30122C0BF75BF0143B40375BB9B43B44A
:104030000475BBABD0BF2290F021E090F003F0906C
:10404000F022E090F002F090F023E090F001F09088
:10405000F024E090F000F090F025E090F007F09070
:10406000F026E090F006F090F027E090F005F09058
:10407000F04DE090F004F00239A3AD07AC06EC126D
:1040800024CAE4FBFA79807843122428E4FBFA7905
:1040900020784202222EE490F0B2F0A3F0123EAA61
:1040A000EF7002FF227F647E19123BE7E490F0B0CC
:1040B000F0A3F090F1161230F890F0B1E09FEE64AA
:1040C00080F890F0B0E0648098506EE0FCA3E0FDD2
:1040D00025E0FFEC33FE74DC2FF974F03EFA7B012F
:1040E000123F2890F0B1E025E0FF90F0B0E033FE01
:1040F00074DC2FF58274F03EF583E0FEA3E0FF113F
:104100007A90F0AC122736E4FFFE7D207C4190F0DF
:10411000AC313C12231F12250390F0B2EEF0A3EF56
:10412000F090F0ECEEF0A3EFF090F0B1E004F0705E
:104130000690F0B0E004F001B37F0122E0F8A3E0C4
:10414000F9A3E0FAA3E0FB22D2051233A500D205C1
:104150001237EE0000000000C2051233A500000077
:104160000000C2050237EE31487FA2319BD2051212
:1041700033A50000000000D2051237EEE4F5B2537B
:1041800086F7000000000030830AC2051237EE12E5
:104190003395C322C2051237EED322E4FE123DFA54
:1041A0005028EF30E704D2058002C2051233A50083
:1041B00000000000D2051237EEEF25E0FF000000FE
:1041C0000000C2051237EE0E80D322300404C2056F
:1041D0008002D2051233A50000000000D20512377C
:1041E000EE0000000000C2051237EED2051233A522
:1041F000000000000022E4F5B25386F7FE123DFAFB
:104200005021D2051237EE0000000000EF25E0FF3C
:104210003083034401FFC2051237EE0000000000A6
:104220000E80DA2212337DEF547FFFEFC4540F75F6
:10423000F00AA4FEEF540F2EFF2212337DEF543FFD
:10424000FF80E87F0112337DEF5408C36001D32261
:10425000EDF090F0A8E0FAA3E0FB7C007D18FFAE43
:1042600002122631A3EEF0A3EFF07C0022E02FFF34
:10427000E43E90F0A6F0A3EFF090F0A6E0FEA3E0FD
:10428000FFE4FCFD7BC07AA8F9F822FDEC4EFEEDC0
:104290004FFF90F0E6EEF0A3EFF022F0A3F0A3F0D2
:1042A000A3F0A3227D18AF03AE02022631E5DD1292
:1042B000260FE5DE541F2290F0ACE075F008A42232
:1042C000C2AF438F0143BB02538FFED2AF22FF9098
:1042D000F0E6E0FCA3E02290F0A6E0FAA3E0FB7C8D
:1042E000007D3C2212259D5403C4333354C0FFE9A2
:1042F00022F9E43AFA02258412340A90F098E02276
:10430000E0FFE4FCFDFE780802270390F0A674A805
:10431000F0A374C0F02275D808E4F5D822E0FF12AB
:1043200036DDEF543FFD22E5DD54FC1313543FFF0F
:01433000226A
:00000001FF
